:10000000BEC00000D7C00000D5C00000D3C00000B3
:10001000D1C00000CFC00000CDC00000CBC00000A8
:10002000C9C00000C7C00000C5C50000C3C00000B3
:10003000C1C00000BFC00000BDC00000BBC00000C8
:10004000B9C00000B7C00000B5C00000B3C00000D8
:10005000B1C00000AFC00000ADC00000ABC00000E8
:10006000A9C00000A7C00000A5C00000A3C00000F8
:10007000A1C000009FC000009DC000009BC0000008
:1000800099C0000097C0000095C0000093C0000018
:1000900091C000008FC000008DC000008BC0000028
:1000A00089C0000087C0000085C000001201100157
:1000B000000000084123370001000102000109028D
:1000C0006500020100C032090400000001010000C7
:1000D00009240100010900010109040100020103D2
:1000E000000007240100014100062402010100066E
:1000F0002402020200092403010301020100092471
:10010000030204010101000905010240000500008D
:1001100005250101010905820240000500000525B1
:1001200001010304030904200353007500730070E8
:1001300000650063007400200044006500760069DB
:1001400000630065007300000032034C006500741A
:100150000027007300200047006500740020004C59
:100160000065006F006E0061007200640020004CAA
:10017000006F00610064006500640000000011244D
:100180001FBECFEFDAE0DEBFCDBF11E0A0E0B1E0EF
:10019000E6E4F1E102C005900D92AA32B107D9F769
:1001A00011E0AAE2B1E001C01D92AF3CB107E1F756
:1001B00002D0C7C725CF1ED020D0FECF0895089506
:1001C000089585E091E0A7C784B7877F84BF88E161
:1001D0000FB6F89480936000109260000FBE80E02C
:1001E00090E020E80FB6F8942093610080936100BE
:1001F0000FBEC3C4E9DF789408951F9385E091E0B2
:100200006DEA71E01BD7882391F08091AD01877072
:1002100081F08091AD018F7082FF0BC06091AD01C4
:100220007091AE018091AF019091B001D7D010E0F4
:1002300001C011E085E091E03FD7EBD6812F1F91FF
:100240000895DA01923049F0933061F09130F9F479
:10025000ECEAF0E022E130E01EC0EEEBF0E025E653
:1002600030E019C0813049F0813018F0823079F4E3
:1002700008C0E3E2F1E0849107C0E7E2F1E0849195
:1002800003C0E9E4F1E08491282F30E004C0E0E00D
:10029000F0E020E030E0ED93FC93C901089511D423
:1002A000F89488E893E120E931E0F9013197F1F71A
:1002B0000197D9F787E797E79093010880930008A3
:1002C0002CE088E190E00FB6F894A8958093600048
:1002D0000FBE20936000FFCFCF93DF938091B401D6
:1002E0008E3731F08F3709F476C08D37F9F419C0A5
:1002F0008091B701863009F06EC08091B8018130DD
:1003000009F069C0C1E1D1E085E091E0BE01E4D629
:10031000249681E0C932D807B9F785E091E0AED6DE
:100320005AC08091B9018E3109F4B9DF10922C01C5
:1003300020E047C080912C01E82FF0E0ED01CC0FC8
:10034000DD1FCC0FDD1FCE54DE4F9981E35DFE4FE4
:1003500090838F5F80932C0188818F70853081F12D
:1003600088818F708F3061F180912C01E82FF0E04F
:10037000AA0FBB1FAA0FBB1FAC54BE4F9C91E35DDD
:10038000FE4F90838F5F80932C0188818F70863021
:10039000B9F088818F708C3099F088818F708D30A2
:1003A00079F088818F70823059F080912C01E82F8C
:1003B000F0E09B81E35DFE4F90838F5F80932C0183
:1003C0002F5FA22FB0E080912A0190912B01A817F6
:1003D000B9070CF4AFCFDF91CF910895CF93DF939E
:1003E0009B01AC01A62FAF706A2F70E0CB01877F15
:1003F000892B09F42AC1A2FF28C18091B101823062
:1004000051F480912A0190912B01813891051CF0C3
:1004100083E08093B1016430710549F06430710567
:100420000CF413C1683071050CF00FC1DCC0809171
:10043000B1018130E9F1813030F0823021F1833037
:1004400009F003C1A8C010922B0110922A01303F7D
:1004500009F0FBC0842F8E57823040F48091000158
:10046000581751F15F3709F0F0C026C080910201A2
:10047000481709F0EAC080910301851709F0E5C02B
:1004800081E08093B10180912A0190912B01FC01C0
:10049000EE0FFF1FEE0FFF1FEE54FE4F2083318340
:1004A00042835383019690932B0180932A01CDC000
:1004B00080910401831711F482E0E3CF83E08093FD
:1004C000B10180912A0190912B01FC01EE0FFF1FD9
:1004D000EE0FFF1FEE54FE4F208331834283538380
:1004E000019690932B0180932A0110922C0120E019
:1004F00047C080912C01E82FF0E0ED01CC0FDD1F0B
:10050000CC0FDD1FCE54DE4F9981E35DFE4F90830B
:100510008F5F80932C0188818F70853081F1888175
:100520008F708F3061F180912C01E82FF0E0AA0FDD
:10053000BB1FAA0FBB1FAC54BE4F9C91E35DFE4F87
:1005400090838F5F80932C0188818F708630B9F003
:1005500088818F708C3099F088818F708D3079F020
:1005600088818F70823059F080912C01E82FF0E063
:100570009B81E35DFE4F90838F5F80932C012F5F03
:10058000A22FB0E080912A0190912B01A817B90702
:100590000CF4AFCF5AC080912C0190E08D379105BB
:1005A0001CF410922C014FC080912C01E82FF0E038
:1005B000E35DFE4F30838F5F80932C0180912C018F
:1005C000E82FF0E0E35DFE4F40838F5F80932C01C6
:1005D00080912C01E82FF0E0E35DFE4F50838F5FA8
:1005E00080932C0132C080912A0190912B01FC0153
:1005F000EE0FFF1FEE0FFF1FEE54FE4F20833183DF
:1006000042835383019690932B0180932A0180911A
:10061000B101823011F460DE16C080912C01E82F08
:10062000F0E0E35DFE4F30838F5F80932C01A530B7
:1006300051F080912C01E82FF0E0E35DFE4F408304
:100640008F5F80932C011092B101DF91CF910895BB
:100650009C014091CD015091CE014617570718F4E7
:10066000F90190E045C06115710511F0AB01F8CFBB
:100670008091E8008E778093E80040E050E0F0CF72
:100680008091C601882309F445C0853009F444C02F
:100690008091E80083FF02C081E008958091E80026
:1006A00082FD32C08091E80080FF22C08091F3007B
:1006B0009091F200782F60E0292F30E0262B372B25
:1006C00007C081918093F100415050402F5F3F4F10
:1006D0004115510519F02830310598F390E0283084
:1006E000310509F491E08091E8008E778093E8006D
:1006F0004115510529F6992319F606C08091C601C6
:10070000882341F0853041F08091E80082FFF6CFE8
:1007100080E0089582E0089583E008959C0140916F
:10072000CD015091CE014617570718F4F90190E01A
:1007300046C06115710511F0AB01F8CF8091E8005A
:100740008E778093E80040E050E0F0CF8091C601C2
:10075000882309F447C0853009F446C08091E80039
:1007600083FF02C081E008958091E80082FD34C0DB
:100770008091E80080FF23C08091F3009091F20007
:10078000782F60E0292F30E0262B372B08C084918A
:100790008093F1003196415050402F5F3F4F4115FB
:1007A000510519F02830310590F390E028303105DB
:1007B00009F491E08091E8008E778093E80041157C
:1007C000510521F6992309F0C1CF06C08091C601D9
:1007D000882341F0853041F08091E80082FFF6CF18
:1007E00080E0089582E0089583E00895BF92CF925B
:1007F000DF92EF92FF920F931F93CF93DF93182F07
:10080000092F7B016A012BD1B82E8823B1F5812FE6
:10081000902F9C01E901C114D10439F0F6018081C7
:100820009181E81AF90AC80FD91F00E010E022C030
:100830008091E80085FD16C08091E8008B77809359
:10084000E800E7D3C114D10449F0F6018081918119
:10085000800F911F9183808385E010C000D1882391
:1008600049F00CC08091F10089930894E108F108E7
:100870000F5F1F4FE114F104D9F68B2DDF91CF915B
:100880001F910F91FF90EF90DF90CF90BF90089550
:10089000BF92CF92DF92EF92FF920F931F93CF936D
:1008A000DF93182F092F7B016A01D9D0B82E882336
:1008B000B1F5812F902F9C01E901C114D10439F0C9
:1008C000F60180819181E81AF90AC80FD91F00E06A
:1008D00010E022C08091E80085FD16C08091E800FC
:1008E0008E778093E80095D3C114D10449F0F601C6
:1008F00080819181800F911F9183808385E010C05A
:10090000AED0882349F00CC089918093F1000894FF
:10091000E108F1080F5F1F4FE114F104D9F68B2DA8
:10092000DF91CF911F910F91FF90EF90DF90CF90CB
:10093000BF900895382F282F2EC0822F8F7080935C
:10094000E900231721F4762F942F50E006C0709110
:10095000EC009091ED005091F00091FF1BC0809150
:10096000EB008E7F8093EB008091ED008D7F809374
:10097000ED008091EB0081608093EB007093EC00C0
:100980009093ED005093F0008091EE0087FD02C03F
:1009900080E008952F5F273080F23F703093E900A8
:1009A00081E008950F931F93CF93DF93062FEC01FF
:1009B00010E02AC09881992329F16B81E981FA819D
:1009C0002C81892F8F70873018F5223010F452E077
:1009D00001C056E040E028E030E003C04F5F220F46
:1009E000331F2E173F07D0F36295660F660F607CAA
:1009F000991F9927991F692B4295407F452B9ADFB4
:100A0000882331F01F5F25961017A0F281E001C006
:100A100080E0DF91CF911F910F9108958091C701E0
:100A200088239CF404C08091C6018823B9F080918A
:100A3000E80082FFF8CF8091E8008B778093E80090
:100A400008958091C601882349F08091E80080FFD5
:100A5000F8CF8091E8008E778093E8000895409168
:100A6000E4005091E50024E68091EC0080FF24C072
:100A70008091E80080FD1EC08091C601882311F49A
:100A800082E00895853011F483E008958091EB00B1
:100A900085FF02C081E008958091E4009091E50017
:100AA0008417950709F3222311F484E00895215057
:100AB000AC01DACF80E008958091E80082FFDCCFBE
:100AC000F9CF6BD072D0E0EEF0E08081816080835E
:100AD000A8EDB0E08C918F778C9319BCE7EDF0E036
:100AE00080818E7F80838C918F7E8C931092C50144
:100AF0000895EF92FF920F931F934FD056D008EDB9
:100B000010E0F80180818F77808380818068808306
:100B100080818F7D808319BC1092C6011092C20122
:100B20001092C4011092C30180EEE82EF12CF7015F
:100B300080818B7F8083F80180818160808380E069
:100B400060E042E0F7DEE1EEF0E080818E7F8083BE
:100B5000E2EEF0E080818160808380818860808324
:100B6000F70180818E7F8083F8018081806180839E
:100B70001F910F91FF90EF900895E8EDF0E08081D4
:100B80008F7E8083E7EDF0E080818160808384E068
:100B900082BF81E08093C501ACCFE8EDF0E08081B9
:100BA0008E7F80831092E20008951092DA001092F6
:100BB000E10008951F920F920FB60F9211242F9308
:100BC0003F934F935F936F937F938F939F93AF93D5
:100BD000BF93EF93FF938091E10082FF0AC0809161
:100BE000E20082FF06C08091E1008B7F8093E100EC
:100BF0000FD28091DA0080FF1DC08091D80080FF65
:100C000019C08091DA008E7F8093DA008091D9003C
:100C100080FF0CC080E189BD82E189BD09B400FE7E
:100C2000FDCF81E08093C601C9DA04C019BC1092DF
:100C3000C601C5DA8091E10080FF18C08091E20012
:100C400080FF14C08091E2008E7F8093E20080914B
:100C5000E20080618093E2008091D80080628093FE
:100C6000D80019BC85E08093C601D2D18091E10003
:100C700084FF2FC08091E20084FF2BC080E189BDFA
:100C800082E189BD09B400FEFDCF8091D8008F7D3F
:100C90008093D8008091E1008F7E8093E100809165
:100CA000E2008F7E8093E2008091E2008160809379
:100CB000E2008091C201882311F084E007C0809196
:100CC000E30087FD02C081E001C083E08093C6019C
:100CD0009FD18091E10083FF22C08091E20083FFD9
:100CE0001EC08091E100877F8093E10082E08093C5
:100CF000C6011092C2018091E1008E7F8093E100D5
:100D00008091E2008E7F8093E2008091E20080611A
:100D10008093E20080E060E042E00CDE79D1FF9158
:100D2000EF91BF91AF919F918F917F916F915F9163
:100D30004F913F912F910F900FBE0F901F901895DC
:100D40001F93DF93CF93CDB7DEB7AC970FB6F89470
:100D5000DEBF0FBECDBFE7ECF1E08091F1008193E3
:100D600021E0EF3CF207C9F72BDA8091E80083FF1E
:100D700037C18091C7013091C801353009F487C06F
:100D8000363040F43130C9F1313070F0333009F091
:100D900027C133C0383009F4F5C0393009F404C133
:100DA000363009F01DC196C0803821F0823809F034
:100DB00017C108C09091C3018091C401882399F0A4
:100DC000926011C08091CB018F708093E900809177
:100DD000EB0090E025E0969587952A95E1F7982F0E
:100DE00091701092E9008091E800877F8093E8007D
:100DF0009093F1001092F100D0C0882319F0823056
:100E000009F0EEC090E08F719070009721F002978A
:100E100009F0E6C00CC08091C901813009F0E0C042
:100E20001092C401333069F58093C4012AC08091C7
:100E3000C901882331F52091CB012F7009F4D0C06E
:100E40002093E9008091EB0080FF1BC0333021F438
:100E50008091EB00806213C08091EB0080618093F1
:100E6000EB0081E090E002C0880F991F2A95E2F71D
:100E70008093EA001092EA008091EB0088608093F2
:100E8000EB001092E9008091E800877F89C08823F9
:100E900009F0A6C01091C9011F778091E300807806
:100EA000812B8093E3008091E800877F8093E800A6
:100EB000B5DD8091E80080FFFCCF8091E300806881
:100EC0008093E300112311F482E001C083E080935A
:100ED000C60186C08058823008F082C08091C90166
:100EE0009091CA0123E08C3D920709F033C083E062
:100EF0008C838AE28B837FB7F894DE0115966EE0CF
:100F000040E050E011E2E62FF0E0109357008491AA
:100F100040FF03C082958F706F5F8F70282F30E085
:100F20008A3018F0C901C79602C0C901C0968D93D6
:100F30009D934F5F5F4F4431510529F77FBF8091EB
:100F4000E800877F8093E800CE0103966AE270E0B4
:100F50007FDB12C06091CB01AE014F5F5F4F71D953
:100F6000BC01009709F43CC08091E800877F809322
:100F7000E80089819A81D2DB8091E8008B778093A9
:100F8000E8002EC0803861F58091E800877F80936B
:100F9000E8008091C2018093F1008091E8008E7793
:100FA0008093E8003BDD1CC08823D1F49091C901F7
:100FB0009230B0F48091E800877F8093E8009093AE
:100FC000C2012CDD8091C201882331F48091E300BD
:100FD00087FD02C081E001C084E08093C601F1D8A2
:100FE0008091E80083FF0AC08091E800877F8093AA
:100FF000E8008091EB0080628093EB00AC960FB626
:10100000F894DEBF0FBECDBFCF91DF911F91089541
:1010100008951F938091C601882371F01091E90013
:101020008091EC001092E9008091E80083FF01C0FC
:1010300087DE1F701093E9001F910895FC018091D5
:10104000C6018430C9F486818F708093E900809155
:10105000E80085FF11C0CB0164E070E040E050E0A3
:10106000C5DB8091E80085FD05C08091E8008B77A5
:101070008093E80081E0089580E00895FC0180916C
:10108000C601843011F082E0089581818F708093D1
:10109000E9004091F3002091F200942F80E030E0CD
:1010A000822B932B892B11F480E008958091E80026
:1010B0008E778093E800D3CCFC018091C601843008
:1010C00051F481818F708093E9008091E80080FF66
:1010D00002C0CF01D3CF0895FC018091C6018430B6
:1010E00011F092E016C081818F708093E900CB01EE
:1010F00064E070E040E050E0CBDB982F882349F4B7
:101100008091E80085FD05C08091E8008E7780938E
:10111000E800892F0895CF93DF93EC011B8682E0CE
:101120008C838987CE01019661E03CDC882331F015
:10113000CE01069661E036DC811181E0DF91CF912E
:061140000895F894FFCFB2
:101146000A0A7D234101824000000101400000019E
:101156000004F07E7F0406027D042341010402019F
:0A11660002040000010621F700005A
:00000001FF
